:1000000000308A0004280000FF238316900000308F
:100010008A00662832308400000803191D28013048
:10002000A100A001A00B1228A10B11284A30A000AA
:10003000A00B18281B28800B0F280800330DA000E8
:10004000A00DFC30A0051F08F33920049F001030DC
:10005000A000A00B29280000B501B401B6013608A4
:100060003F3C031C53289F1437109F1C371437182C
:100070003D2837109F1C371437289F183D281E082D
:10008000A30083161E088312B8001E08B9003808A2
:10009000A1003908A2002108B40722080318220F82
:1000A000B507B60A2F28B50CB40CB50CB40CB50CBA
:1000B000B40CB50CB40CB50CB40CB50CB40C0330CA
:1000C000B5053408A1003508A200080084011F30DE
:1000D00083051F1383161F109F101F119F110730D8
:1000E000831299000F308316850083128512051242
:1000F00083161F169F121F1383129F171F141F139F
:1001000083161F149F141F159F118312AB01AA01A0
:10011000A9012B0803199628013A0319CC28033AA0
:100120000319F828013A03196E299A29B001AF0181
:10013000AE01AD01AA01A90105166430B2000A2082
:100140000230B3001E202208A6002108A500B3013A
:100150001E202208B2002108B1000130B3001E2089
:1001600021083102A7003208A8002208031C220F30
:10017000A802A608031DC02825080F3C0318C328A1
:100180000130AB00CB2805120430B100E130B200E1
:100190000A20B10BC6289C2905160130AD070318AB
:1001A000AE0A0319AF0A0319B00AB008031DE62806
:1001B000AF08031DE6282E080A3C0318E928FF3A79
:1001C000031DE6282D08B73C0318E9280230AB00D0
:1001D0009C290230B3001E202208A6002108A50099
:1001E000A608031DF72825080E3C0318AB019C291F
:1001F00005160130AD070318AE0A0319AF0A03193B
:10020000B00A0230B3001E202208A6002108A50073
:10021000B3011E202208B2002108B1000130B30052
:100220001E2021083102A7003208A8002208031C62
:10023000220FA802A608031D232925080E3C031C33
:100240002329AB019C292808013C03183029FF3AD7
:10025000031D2E292708BB3C03183029AB019C291C
:10026000B008031D45292F08003C03184829FF3A10
:10027000031D45292E08503C03184829FF3A031D49
:1002800045292D08803C031848290330AB009C29E0
:100290002A082802031C5629031D5229270829026F
:1002A000031856292808AA002708A90001302902A6
:1002B000A0002A08A3000030031C0130A30220087C
:1002C000A10028082302031C6D29031D6B292108A6
:1002D000270203186D290330AB009C29B001AF0140
:1002E000AE01AD01AA01A90105120830B100FA3032
:1002F000B2000A20B10B7729B3011E202208B200F8
:100300002108B1000130B3001E2021083102A700EE
:100310003208A8002208031C220FA8022808013C6A
:1003200003189929FF3A031D98292708BB3C031C91
:10033000AB019C29AB019C296430B2000A202B0838
:100340000319AC29013A0319AE29033A0319B0295C
:10035000013A0319C629C8298512C9298516C92950
:100360002D080239A000A101A201A301A008031DCC
:10037000C229A108031DC229A208031DC229A3087E
:100380000319C4298516C5298512C9298516C929C5
:06039000C9298928630061
:02400E00443F2D
:00000001FF
